:100000000C9493020C94CB020C94CB020C94CB0274
:100010000C94CB020C94CB020C94CB020C94CB022C
:100020000C94CB020C94CB020C944D0D0C948F0CC1
:100030000C94031A0C94CB020C94CB020C94CB02BC
:100040000C94CB020C94CB020C94CB020C94CB02FC
:100050000C94CB020C94C5190C94CB020C94CB02DB
:100060000C94CB020C94CB020C94CB020C94CB02DC
:100070000C94CB020C94CB020C94CB020C94CB02CC
:100080000C94CB020C94CB020C94CB020C94CB02BC
:100090000C94CB020C94CB020C94CB020C94CB02AC
:1000A0000C94CB020C94CB020C94CB026C05E005B3
:1000B00074053E054205780545057B058605500516
:1000C000D60554058A0558058E05B8055C059205C8
:1000D000C20562059805A20549057F054C05820504
:1000E00067059D05AE05CE05D0053A057005E90505
:1000F0000F061506030609061B0621062706CA0673
:10010000CA06FD06FD06770798089808980895071F
:1001100009081A081A08A70ACE0A770CCE0A770C23
:100120001A0B3D0B770C320C420CED15F0151B161B
:100130002B1632163D16DA16DA16DA16DA16DA1633
:100140004016421647166D16901693169616BA1656
:10015000000000000000000000000000000000009F
:10016000000000000000000000000000000000008F
:10017000000000007E0F00D4FFFFFFC700000078E2
:1001800000000000000000002A2B280000000000F2
:100190000000000000000000000000290000000036
:1001A0002C1E3420212224342627252E362D3738A4
:1001B000271E1F202122232425263333362E3738AD
:1001C0001F0405060708090A0B0C0D0E0F1011126B
:1001D000131415161718191A1B1C1D2F3130232D37
:1001E000350405060708090A0B0C0D0E0F10111235
:1001F000131415161718191A1B1C1D2F3130354CE6
:1002000005010980A101850319012AB700150126FE
:10021000B700950175108100C0050C0901A1018589
:100220000419012AA002150126A00295017510816A
:1002300000C005010906A1018506050719E029E7A7
:10024000150025019508750181020507190029EFA0
:100250001500250195F07501810205081901290590
:10026000950575019102950175039101C00660FF26
:100270000961A1010962150026FF0095207508811A
:10028000020963150026FF00952075089102C0053C
:10029000010906A101050719E029E71500250195C7
:1002A000087501810295017508810105071900296A
:1002B000FF150026FF009506750881000508190145
:1002C0002905950575019102950175039101C009F4
:1002D000025B00030100A0FA090400000103010110
:1002E00000092111010001224000070581030800D7
:1002F00001090401000203000000092111010001AD
:1003000022220007058203200001070503032000C5
:10031000010904020001030000000921110100018C
:10032000226D000705840320000112010002000075
:10033000000868616670000101020001240370007A
:10034000690061006E006F0066006F00720074004B
:100350006500200073006F006C006400650072008F
:1003600000000E0341006C00690063006500480056
:1003700000000403090429003B003D003F00410048
:1003800043004500460048003A003C003E00400063
:100390004200440068004700000035001F002100B3
:1003A0002300250027002E002A004A001E002000FE
:1003B0002200240026002D002A00490000004B00E6
:1003C000140008001700180012002F0031004D0023
:1003D0002B001A0015001C000C00130030004C000C
:1003E00000004E00040007000A000D000F0034005A
:1003F000280000003900160009000B000E00330031
:10040000320000000000E1001D00060005001000A1
:100410003700E5005200000064001B0019001100C5
:1004200036003800E500E0000000E3002C0000008A
:10043000000000000000215250004F00E2000000C8
:10044000000021520000E700E4005100000001001C
:100450000100010001000100010001000100010094
:100460000100010001000100010001000100010084
:100470000000010001000100010001000100010075
:100480000100010001000100010001000100010064
:100490000100010000000100010001000100010055
:1004A0000100010001000100010001000100010044
:1004B0000100010001000100000001000100010035
:1004C0000100010001000100010000000100010025
:1004D0000100010001000100010000000000010016
:1004E0000100010001000100010001000100000005
:1004F00001000100010001000100010001000100F4
:1005000000000100010000000000000000000100E8
:1005100001000100010000000000010000000100D6
:1005200001000100000011241FBECFEFDAE0DEBFA2
:10053000CDBF04B603FE18C080919B0290919C022F
:10054000A0919D02B0919E028730904BA740B04B86
:1005500059F410929B0210929C0210929D021092EC
:100560009E02E0E0F8E3099511E0A0E0B1E0E2EAE4
:10057000F9E302C005900D92A236B107D9F722E047
:10058000A2E6B1E001C01D92AB39B207E1F70E94CB
:10059000AC130C94CF1C0C9400000E94FD172FE7A5
:1005A0008AE196E0215080409040E1F700C00000D1
:1005B0009CE088E10FB6F894A895809360000FBE88
:1005C00090936000FFCFA7E1B0E0E9EEF2E00C9479
:1005D0009A1C4B8B5C8B6D8B7E8B8F8B6111109279
:1005E000100286E09E01235F3F4FD901E82F1D9244
:1005F000EA95E9F795E0FE017396D90101900D9215
:100600009A95E1F79C894E895F897B897D879E87D2
:100610006F87598B488BF901DE01179601900D9277
:100620008A95E1F7CE0107960E94251281113EC0FE
:1006300086E0FE013796DE01119601900D928A95B3
:10064000E1F7FF81E8856A857B856115710531F0E9
:10065000EF3F31F481E0FF3F19F403C081E001C0B6
:1006600080E080FD23C02091BD0130E0C9010196EA
:10067000877099274091EE0150E08417950779F132
:10068000F983EA837D836C8396E0929FD001939FE8
:10069000B00D1124A254BE4FFE01319601900D926F
:1006A0009A95E1F78093BD010E94B21116E0809106
:1006B000EE019091BD018917F9F0189FC001112436
:1006C00082549E4F0E9425128823B1F08091EE0142
:1006D00090E00196877099278093EE01E8CF0E9401
:1006E000FD171092BD011092EE01E7EBF1E086E0FC
:1006F000DF011D928A95E9F76796E3E00C94B61C3A
:10070000ADE0B0E0E6E8F3E00C948B1CFC018081E6
:10071000918123813481232B31F09F3F31F491E08B
:100720008F3F19F403C091E001C090E090FD3EC5F9
:100730007F0185E0DE01199601900D928A95E1F71F
:10074000F701228189859A85222349F00E940217A8
:10075000182F682F89859A850E94721703C00E94FE
:100760003E17182F69857A85812F0E94700F8C01A2
:10077000F7018281882309F42CC198012250374760
:100780002031310508F041C18FEF93E00E943C1CFD
:10079000811129C1025036EDA32EBB24B39400234E
:1007A00079F0A114F4E0BF0609F41DC1C5010E944F
:1007B0003C1C811101C001502FEFA21AB20AEFCFE9
:1007C000CE0101962C0188E0F20111928A95E9F799
:1007D0002AE0322E85010F5F1F4FC5010E943C1C8D
:1007E00089831A82882309F4FEC0813009F041C050
:1007F0006501F2E0CF0ED11CC8010E943C1C8A8327
:10080000882309F4F0C09FEF980F933060F423E041
:10081000A20EB11CC6010E943C1C8B83882309F4E4
:10082000E2C01C8229C0843031F54E0133E0830ED2
:10083000911C02E010E056018FEFA81AB80AC60119
:100840000E943C1CF40181934F01882309F4CBC022
:100850008C3741F4E2E0F0E0EC0FFD1FE00FF11FF8
:1008600010820AC00F5F1F4F65010730110519F78D
:10087000BAC0580101C056018201F801208122232B
:1008800009F4A8CF213009F04CC08181813049F4AE
:100890006801F2E0CF0ED11CF80182810E9441195B
:1008A0000AC0823051F46801F2E0CF0ED11CF80189
:1008B00082810E948718860189C0833049F46801CB
:1008C000F2E0CF0ED11CF80182810E942E18F3CFE6
:1008D000843019F00F5F1F4F79C0F80122810E5F3D
:1008E0001F4F80E090E030E0205331092A3031057D
:1008F00068F4389EA001399E500D1124C901840F5F
:10090000951F0F5F1F4FF8012081EDCF009709F46D
:100910005DC0EFECF7E03197F1F700C00000019700
:10092000F5CFE22FF0E0E058FE4F2490822F86951D
:100930008695869590E0FC01E059FE4F6490277003
:10094000712C022E02C0759467940A94E2F7F1E0CC
:100950006F227724FC01E05AFE4F8490912C022EE6
:1009600002C0959487940A94E2F731E08322992497
:10097000FC01E05BFE4FC490D12C02C0D594C7941B
:100980002A95E2F781E0C822DD246114710419F090
:1009900081EE0E9487188114910419F086EE0E945E
:1009A0008718822D0E9441198114910419F086EE56
:1009B0000E942E186114710419F081EE0E942E1805
:1009C000C114D10419F08CE20E9441190F5F1F4F2E
:1009D00054CF011537E7130709F042C181E00E94A7
:1009E000AA170E94B8098091EF01877009F4DEC34D
:1009F000F7018281882309F4D9C38091660182FFBF
:100A0000D5C382E00E947E11D1C30115F7E71F070D
:100A100011F481E005C0013027E7120721F482E0DC
:100A20000E94B717DECFF801E851FC47E730F10527
:100A300008F4E5C0882309F45BC110928F02C80155
:100A40009057839708F013C184E090E00E94441C03
:100A50009093660180936501F801E150F047E2321E
:100A6000F10520F4EA5AFF4F0C947E1C8091650139
:100A70008160ACC0809166018860B4C080916501DE
:100A80008260A4C08091650120C08091650188606A
:100A90009DC0809166011EC0809166018260A2C0E7
:100AA00080916501806192C08091650180628EC0F5
:100AB0008091650180648AC00E94FD178091650164
:100AC000806884C080916501886084607FC0809167
:100AD00066018260816086C0809165018E7F76C0EC
:100AE00080916601877F7EC0809165018D7F6EC099
:100AF0008091650120C080916501877F67C08091EA
:100B000066011EC0809166018D7F6CC08091650179
:100B10008F7E5CC0809165018F7D58C0809165019A
:100B20008F7B54C00E94FD17809165018F774EC066
:100B300080916501877F8B7F49C0809166018D7FA1
:100B40008E7F50C08091650182FB222720F991E0C1
:100B5000922790FB82F990FB83F938C0809166015F
:100B6000982F909591708E7F892B90FB81F93AC0D8
:100B70008091650186FB222720F991E0922790FB66
:100B800086F924C00E94FD178091650187FB22270A
:100B900020F991E0922790FB87F918C061E001C02D
:100BA00060E08EE090E00E944A1C1EC080916501CA
:100BB00084FB222720F991E0922790FB84F906C05C
:100BC00080916501982F909590FB80F98093650145
:100BD0000BC08091660183FB222720F991E09227C8
:100BE00090FB83F9809366016091650170916601C5
:100BF00084E090E00E94681C0E94FD17F4CEE85843
:100C0000FF4F0C947E1C06E221EE41EE6AE17CE788
:100C100023C007E225EE45EE6BE17CE71DC006E24E
:100C200021EE40EE68E17CE717C007E225EE44EED6
:100C300069E17CE711C006E221EE42EE6CE17CE75F
:100C40000BC007E225EE46EE6DE17CE705C008E249
:100C500021E045EE6EE17CE7C7010E94E01AC3CEB9
:100C6000013097E7190709F0DECE82E0B8CE0631F1
:100C7000ECE71E0709F47AC203309CE7190721F15B
:100C800040F40115FCE71F0789F001301C4711F102
:100C900034C00B353CE7130739F10C358CE71807E6
:100CA000D9F00A351C4749F581E01FC00E94FD17A5
:100CB000EFE7FAE126E0E150F0402040E1F700C024
:100CC00000000E94A1198FCE6FEF7FEF80E090E0CF
:100CD0000E94681C0E94CD028091660182FB8827D9
:100CE00080F991E0892701C080E00E949B1105C036
:100CF0000631FCE71F0709F449C2F7018281008130
:100D00001181882349F0C8010E940217D82E682F4C
:100D1000C8010E94721704C0C8010E943E17D82E55
:100D2000B8018D2D0E94700F0E947E0FB82E192FD2
:100D3000982EF7010281A580A2949FE0A9228091BC
:100D4000EF018770B9F00023A9F0812F807F8034F4
:100D500021F080E28B0D883068F08091660182FF7F
:100D600009C082E00E947E118091EF018770DD242E
:100D7000D3948111D12CC12EC2948FE0C8228C2D26
:100D800090E08C30910508F0D3C1FC01E158FF4F91
:100D90000C947E1C812F807F1F70882311F0129588
:100DA000107F0023B9F0112309F4B0C180E28B0D4C
:100DB000883010F0911006C090911102192B1093F9
:100DC000110205C090911002192B109310020E947D
:100DD00029119CC18B2D0E942E18112309F4A8C142
:100DE00080E28B0D883088F1992079F110959091EF
:100DF00010021923109310022BC0812F807F1F70C7
:100E0000803211F01295107F8B2D992029F0F1E09E
:100E10009F1609F441C04FC08091660182FD1BC03E
:100E2000002369F0112339F090911102192B1093CE
:100E300011020E94291180E00E94871879C180E088
:100E40000E942E18112309F473C1812F0E942211D0
:100E50000E9429116DC1002381F080911202AA2005
:100E600051F021E0A21207C0182B181709F460C135
:100E7000109312025DC1812B16C0A11003C00E9405
:100E80001C1131C031E0A31609F452C1812F0E9418
:100E90001D180E941C114CC1002341F085E08A15E9
:100EA00008F446C1812F0E94241842C194E09A158B
:100EB00008F43EC118C0002349F0AA2099F3F701B5
:100EC000858180FF23C18F708583ECCFAA2059F0E4
:100ED000893309F02AC1FFEF23EF31E0F1502040C0
:100EE0003040E1F720C1812F0E941D1821C1812FC0
:100EF00086958695837019F0813061F019C10023C1
:100F000021F08B2D912F937002C080E090E00E9421
:100F1000AE1A14C1002321F08B2D912F937002C0C3
:100F200080E090E00E94891A09C1812F8370A9F5A1
:100F3000011102C14B2D429546954770440F440F55
:100F40008B2D8F7090E09C01042E01C0220F0A941B
:100F5000EAF7B4FE08C08FE090E001C0880F4A9520
:100F6000EAF7809501C080E016951695137012304F
:100F700069F088F490912E02113019F0822B8923A8
:100F800002C0922B892B0E94C317D6C0822B90914E
:100F90002E028927F8CF822BF6CF002319F0812F5C
:100FA000817001C08695882309F4C6C04B2D4295F7
:100FB00046954770440F440F8B2D8F7090E09C0135
:100FC000042E01C0220F0A94EAF7B4FE08C08FE095
:100FD00090E001C0880F4A95EAF7809501C080E053
:100FE000169516951370123059F078F49091960179
:100FF000113019F0822B892309C0922B892B06C04E
:10100000822B90919601892701C0822B0E94A717FD
:1010100093C01F70002339F0812F0E94B7178B2DCA
:101020000E94241889C08B2D0E941D18812F0E94B8
:10103000AA1782C08B2D92EF991681F1991538F07D
:10104000E0EF9E1659F0F1EF9F1619F15BC023EF08
:10105000921659F134EF9316C1F054C0002381F079
:1010600084E08A1508F464C01F7181E090E0012ECD
:1010700001C0880F0A94EAF790919601892720C051
:1010800095E09A1508F454C0EFCF8091660182FD77
:101090001AC0002329F0812F8F7127C00023D9F3B4
:1010A000812F8F710E94AA1743C0002341F01F7146
:1010B00081E0012E01C0880F0A94EAF701C080E0A8
:1010C0000E94A71735C0002399F01F71812F0E943D
:1010D000B7178091660182FF07C0E8E01E9FC0013C
:1010E000112483608093EF01812F0E94B71720C0E5
:1010F00081E00E947E11F1E0FA15D0F482E00E94B6
:101100007E1116C0002321F0AA2029F28B2D94CE47
:10111000AA2031F2893349F42FEF33EF81E02150D7
:1011200030408040E1F700C000008B2D0E942E1857
:1011300088EF8C0D843010F40E94D31ADD20B1F1B9
:101140008091EF0180FD32C0F7011282859585956F
:1011500085950E94B717C7010E9480038091EF0117
:101160008595859585950E94AA1720C080911102CA
:101170008A7A91E009F490E090936401811112C0A1
:1011800069E287E991E00E94541A09C080916401E4
:1011900081110AC069E287E991E00E942C1A0E943D
:1011A000291121CC65E3EDCF65E3F5CF2D96E2E182
:1011B0000C94A71C80918E0187FF11C08091E800DC
:1011C00082FD05C080918C018111F8CF11C0809102
:1011D000E8008B770BC080918C01882349F08091C7
:1011E000E80080FFF8CF8091E8008E778093E800D8
:1011F0000895982F973068F59093E900981739F083
:101200007091EC002091ED005091F00003C0242F6C
:10121000762F50E021FD02C09F5FECCF3091EB00B4
:101220003E7F3093EB003091ED003D7F3093ED0039
:101230003091EB0031603093EB007093EC00209321
:10124000ED005093F0002091EE0027FDE5CF80E007
:1012500008958F708093E90081E0089520919401B2
:10126000309195012617370748F06115710539F45B
:101270002091E8002E772093E80001C0B901FC011D
:1012800020E06115710579F180918C018823F1F1DD
:101290008530F1F18091E80083FD3CC08091E80049
:1012A00082FD2EC08091E80080FFEBCF2091F300FB
:1012B0008091F20090E0922B6115710551F0883019
:1012C000910538F421912093F10061507109019644
:1012D000F3CF21E0089709F020E08091E8008E77B5
:1012E0008093E800CECF2111CFCF0AC080918C012E
:1012F000882361F0853061F08091E80083FD0AC0A9
:101300008091E80082FFF2CF80E0089582E00895A6
:1013100083E0089581E00895089543E050E0BC0122
:1013200084E00E9463190895CF93DF93EC018091CC
:101330000001811105C048E050E0BE0181E00BC012
:101340008091650187FF03C040E284E002C048E06D
:1013500081E050E0BE010E94631980E2FE01AAE62E
:10136000B1E001900D928A95E1F7DF91CF91089558
:1013700080919601982F9670963011F4886001C084
:10138000877F0E94A7170895AAE2B0E0EAECF9E08F
:101390000C949A1CEEE8F1E086E991E02091F100CE
:1013A00021938E179F07D1F780918F01833009F425
:1013B00063C030F4813071F0823009F49DC0B4C054
:1013C0008A3009F489C08B3009F46EC0893009F085
:1013D000ABC020C080918E01813A09F0A5C08091F8
:1013E000E800877F8093E8008091920190919301BB
:1013F000892B21F460E28AE691E003C060E080E09E
:1014000090E070E00E942E098091E8008B77809335
:10141000E8008AC080918E01813209F085C08091F8
:10142000920190919301009719F0029709F07CC006
:101430008091E800877F8093E8008091E80082FD3A
:1014400005C080918C018111F8CF6EC02091F3000E
:101450008091F20090E0922B029731F48091F1009C
:10146000813011F0863021F48091F1008093690180
:101470008091E8008B7754C080918E01813A09F009
:1014800053C08091920190919301892B09F04CC037
:101490008091E800877F8093E8008091E80080FFDA
:1014A000FCCF8091000137C080918E018132E1F53F
:1014B0008091920190919301892BB1F58091E80080
:1014C000877F8093E8000E94DA08809190018093E2
:1014D00000010E94FD1728C080918E01813221F504
:1014E0008091E800877F8093E8000E94DA0880916D
:1014F00091018093680118C080918E01813AA1F416
:101500008091E800877F8093E8008091E80080FF69
:10151000FCCF809168018093F1008091E8008E7784
:101520008093E8000E94DA088091E80083FFDFC121
:1015300080918E0190918F01492F50E04A305105E2
:1015400008F0D5C1FA01E557FF4F0C947E1C803896
:1015500021F0823809F0CBC108C080918A019091B6
:101560008B01992389F082600FC0809192018F7066
:10157000873008F0BCC18093E9008091EB0085FBC7
:10158000882780F91092E9009091E800977F909366
:10159000E8008093F1001092F10070C1282F2D7F98
:1015A00009F0A5C1882319F0823061F0A0C18091B3
:1015B0009001813009F09BC1933009F080E0809365
:1015C0008B012EC08091900181112AC080919201DF
:1015D0008F702FEF280F263008F089C18093E90023
:1015E0002091EB0020FF1CC0933021F48091EB0090
:1015F000806214C09091EB0090619093EB0021E029
:1016000030E0A90102C0440F551F8A95E2F74093CC
:10161000EA001092EA008091EB0088608093EB0072
:101620001092E9008091E800877F8093E8000E9493
:10163000DA085DC181115BC1109190011F77809123
:10164000E3008078812B8093E3008091E800877F1E
:101650008093E8000E94DA088091E80080FFFCCFC8
:101660008091E30080688093E300111102C082E062
:1016700001C083E080938C013AC18058823008F029
:1016800036C120919001309191012C3D53E03507F6
:1016900079F583E08A838AE289834FB7F894DE0183
:1016A000139620E03EE051E2E32FF0E05093570024
:1016B000E49120FF03C0E295EF703F5FEF708E2F43
:1016C00090E0EA3010F0C79601C0C0968D939D93CC
:1016D0002F5F243149F74FBF8091E800877F8093C7
:1016E000E8006AE270E0CE0101960E942E09B4C0C3
:1016F0008091920190919301432F552743305105DA
:10170000A9F068F44130510509F400C14230510597
:1017100009F0EDC08BE590E0EFECF2E04BC0413218
:10172000510529F14232510589F1E1C0C9019927DA
:1017300081309105A1F058F0029709F0D8C0ECE390
:10174000F3E0E4918E2F90E0ECE3F3E030C0E2E7C9
:10175000F3E0E4918E2F90E0E2E7F3E028C0E2E6C8
:10176000F3E0E4918E2F90E0E2E6F3E020C08330D6
:10177000910508F0BCC0880F991FFC01EE5EFE4F7A
:101780000190F081E02D89E090E014C08330910554
:1017900008F0ADC0FC01EE0FFF1FE45FFE4F0190AB
:1017A000F081E02DDC01A75FBE4F8C9190E00097A7
:1017B00009F49DC02091E800277F2093E800209144
:1017C0009401309195012817390708F4C90140E0C8
:1017D000009789F120918C01222309F43DC0253026
:1017E000D9F12091E80023FD37C02091E80022FDC7
:1017F0002FC02091E80020FFEBCF4091F300209113
:10180000F20030E0342B009759F02830310540F4D5
:1018100044914093F100319601972F5F3F4FF3CFF2
:1018200041E02830310509F040E02091E8002E77B2
:101830002093E800CDCF4111CDCF0AC080918C011B
:10184000882351F0853041F08091E80083FD04C089
:101850008091E80082FFF2CF8091E8008B7780933F
:10186000E80045C0803809F042C08091E800877FD9
:101870008093E80080918D018093F1008091E800D1
:101880008E77D3CE811133C08091900190919101D8
:101890009927029764F58091E800877F8093E8009C
:1018A0001091900110938D010E94DA08111106C069
:1018B0008091E30087FD02C081E001C084E0809355
:1018C0008C0142E061EC81E00E94F90842E261ECA7
:1018D00084E00E94F90842E261EC82E00E94F9088B
:1018E00042E260EC83E00E94F90880918C018091D3
:1018F000E80083FF10C08091E800877F8093E800B4
:101900008091EB0080628093EB0005C082E190E063
:10191000EAE2F3E04FCFAA96E3E00C94B61C1F92E4
:101920000F920FB60F9211242F933F934F935F9313
:101930006F937F938F939F93AF93BF93CF93DF93D7
:10194000EF93FF93C091E900CF708091EC00D82F06
:10195000D17080FDD0E81092E9008091F000877F7F
:101960008093F00078940E94C4091092E90080915D
:10197000F00088608093F000CD2BCF70C093E90019
:10198000FF91EF91DF91CF91BF91AF919F918F9197
:101990007F916F915F914F913F912F910F900FBE6B
:1019A0000F901F901895E8EDF0E080818E7F808386
:1019B0001092E2001092DA001092E100A0EEB0E086
:1019C0008C9181608C9380818F77808319BCA7ED87
:1019D000B0E08C918E7F8C9380818F7E808310927B
:1019E00067010895A0E0B0E0E8EFFCE00C94951CDE
:1019F000C8EDD0E088818F7E8883E7EDF0E08081BC
:101A00008160808384E082BF81E080936701888168
:101A10008E7F888302EE10E0F80110821092DA00C7
:101A200081EEC82ED12CF601108288818F778883B1
:101A300088818068888388818F7D888319BC109213
:101A40008C0110928D0110928B0110928A0190EE00
:101A5000E92EF12CF70180818B7F80838881816062
:101A6000888342E060E080E00E94F908F60180810E
:101A70008E7F8083F801808181608083808188608F
:101A80008083F70180818E7F808388818061888355
:101A9000CDB7DEB7E8E00C94B11C1F920F920FB6E1
:101AA0000F9211242F933F934F935F936F937F93E4
:101AB0008F939F93AF93BF93EF93FF938091E10038
:101AC00082FF09C08091E20082FF05C08091E100A1
:101AD0008B7F8093E1008091DA0080FF28C08091A5
:101AE000D80080FF24C08091DA008E7F8093DA00D6
:101AF0008091D90019BC80FF16C082E089BD09B46D
:101B000000FEFDCF81E080938C01809167018111FF
:101B10000EC00E94D30C0E94F20C8091E2008460FF
:101B20008093E20004C010928C01109267018091B2
:101B3000E10080FF17C08091E20080FF13C0809118
:101B4000E2008E7F8093E2008091E20080618093CA
:101B5000E2008091D80080628093D80019BC85E0B3
:101B600080938C018091E10084FF2FC08091E2007E
:101B700084FF2BC019BC82E089BD09B400FEFDCFF3
:101B80008091D8008F7D8093D8008091E1008F7E76
:101B90008093E1008091E2008F7E8093E20080914B
:101BA000E20081608093E20080918D01882311F032
:101BB00084E007C08091E30087FD02C081E001C09E
:101BC00083E080938C0180918C018091E10083FF00
:101BD00027C08091E20083FF23C08091E100877FCE
:101BE0008093E10082E080938C0110928D018091BE
:101BF000E1008E7F8093E1008091E2008E7F8093F0
:101C0000E2008091E20080618093E20042E060E0C7
:101C100080E00E94F9088091F00088608093F000D5
:101C2000FF91EF91BF91AF919F918F917F916F91B4
:101C30005F914F913F912F910F900FBE0F901F908A
:101C400018952091E4003091E50095E64091EC0074
:101C5000842F817040FF23C08091E80080FD1DC06B
:101C600080918C01882399F0853099F08091EB0068
:101C700085FD11C04091E4005091E500241735071F
:101C800029F3915011F09A01E1CF84E0089582E0A8
:101C9000089583E0089581E0089580E008954091DB
:101CA000E80042FFDDCF089580E00895909165013E
:101CB00092FF0DC0282F2871283019F4877F846087
:101CC00006C0282F2471243011F48B7F886093FF85
:101CD0000DC0282F2871283119F4877E846106C031
:101CE000282F2471243111F48B7E886120916601A4
:101CF00020FF0DC0382F3871383019F4877F81608C
:101D000006C0382F3171313011F48E7F886021FF89
:101D10000DC0282F2871283119F4877E816106C0F3
:101D2000282F2171213111F48E7E886194FD877EE8
:101D30000895F894E82FE295EF70F0E031A1282F94
:101D40002F7081E090E001C0880F2A95EAF7982F64
:101D50009095932391A392A1892B82A378940895BF
:101D6000A8E1B0E0E6EBFEE00C948D1CAE014F5F05
:101D70005F4F7A0188E1FA0111928A95E9F70DE443
:101D800011E06A0199E5492E91E0592E6624639489
:101D9000712C32E6832E31E0932EF80180818F3F43
:101DA00009F446C0F894E82FE295EF70F0E021A125
:101DB0008F70A30102C0440F551F8A95E2F7CA0134
:101DC000922F982B91A392A18095892382A3789436
:101DD00000C0E9E5F1E021E030E0A12CB12C419117
:101DE0004F3F89F0A42FA295AF70B0E090968C91F0
:101DF00090E04F7002C0959587954A95E2F780FD77
:101E000002C0C90102C080E090E0A82AB92A220FCE
:101E1000331F8E169F0619F7F80180818F3F11F04E
:101E20000E94990EF0E5FA95F1F7F601B182A082D1
:101E30000F5F1F4FF2E0CF0ED11C4016510609F084
:101E4000ACCF48E150E0B70186E192E00E94C21CAD
:101E5000892B89F088E1F701A6E1B2E001900D92AB
:101E60008A95E1F781E0809315020E94F71990931B
:101E700014028093130280911502811102C080E048
:101E80002BC020911302309114024FB7F894809127
:101E9000970290919802A0919902B0919A024FBF37
:101EA000821B930B059758F348E150E066E172E01E
:101EB0008BE492E00E94C21C892B59F088E1E6E194
:101EC000F2E0ABE4B2E001900D928A95E1F781E097
:101ED00001C080E0109215026896E0E10C94A91C04
:101EE0007C3048F4693038F4823028F4462F672F6C
:101EF0000E94C11B089580E090E00895CF93DF9386
:101F00008238910569F1B0F48133910509F477C005
:101F100048F48932910509F469C08A32910509F4BF
:101F200073C092C08533910509F45BC08933910574
:101F3000B9F08AC0833E910591F138F4803E910555
:101F4000D1F0823E910531F17FC0863E9105D9F1F5
:101F5000873E9105E9F1843E910509F075C028C0DE
:101F60002091650120FD5BC021FD59C020916601D3
:101F700023FD61C069C08091650180FD4AC08091E8
:101F8000660180FF4CC08091650184FD50C183EEE5
:101F900090E04FC18091650182FF3EC0F4CF8091F7
:101FA000650182FD39C08091660180FD38C0EBCFAC
:101FB0008091660181FF39C08091650184FD37C140
:101FC00087EE90E036C18091650183FF2BC0F4CF8E
:101FD0008091650183FD26C08091660181FD25C049
:101FE000EBCF8091650185FD26C022C080916501FF
:101FF00085FD1EC08091660183FF1DC00AC08091CF
:10200000650186FD1BC01DC08091650186FD19C05C
:1020100015C089E390E00DC182EE90E00AC180EE28
:1020200090E007C186EE90E004C184EE90E001C12B
:1020300085E390E0FEC089E290E0FBC08AE290E098
:10204000F8C081E390E0F5C0EC01811530E593071D
:1020500008F053C0811560E4960720F0CE019F7010
:10206000906AE7C0803E910588F58D3C910518F097
:10207000CE019065DEC0883A9105C0F4853A91059D
:1020800050F08C2F855AC82FD0E0C85EDE4F888173
:1020900090E09064CEC08130910509F4C5C008F489
:1020A000C6C0049708F4C3C0CE01C3C0813C9105EB
:1020B00008F0BDC08C2F885AC82FD0E0CC0FDD1F90
:1020C000C55EDE4F888199819464B3C081159042CA
:1020D00058F08D2F8F710E94560E282F2F71CE0130
:1020E00099279062922BA5C0C11581E0D807E0F630
:1020F000C83ED10508F09BC0D7CFC03692E5D907BE
:1021000008F053C0C03422E5D207B8F08C2F8F718D
:102110008695869570E2879FA00111248C2F83708D
:1021200021E030E0B90102C0660F771F8A95E2F71F
:10213000CB019C68842B952B7CC0C03232E5D30741
:1021400040F08C2F8F7190E0982F8827816F906AD4
:1021500070C0C11562E5D607B0F08C2F86958695C4
:1021600020E2829FA00111248C2F837021E030E0B7
:10217000B90102C0660F771F8A95E2F7CB01842B65
:10218000952B9D6856C08C2F8F710E94560E95E03E
:10219000D695C7959A95E1F7CF70D0E0DC2FCC2784
:1021A000D0699E01282BC90144C0C03A72E5D70707
:1021B00008F58C2F8F71C03892E5D907A8F4869561
:1021C000869570E2879F900111248C2F837041E0E7
:1021D00050E0BA0102C0660F771F8A95E2F7CB0183
:1021E0009A68822B932B25C090E0982F8827846FC4
:1021F000906A1FC0C03C22E5D20750F48C2F8F712B
:102200000E94560E8F7190E0982F8827906211C01F
:10221000C03E32E5D30758F4CE018F719927982F2D
:102220008827806F906A05C081E090E002C080E05E
:1022300090E0DF91CF910895809112028111109268
:1022400012020895809590911102892380931102C2
:1022500008959091110280911002982B909397010C
:10226000809112028823D9F0892B80939701809165
:102270000001882331F08091650187FF02C08EE163
:1022800001C086E0E9E9F1E090E0815028F0219179
:102290002223D9F39F5FF9CF91110E941C1140E2D4
:1022A00050E060EF71E087E991E00E94C21C892B49
:1022B00021F180E2E7E9F1E0A0EFB1E001900D92B9
:1022C0008A95E1F7E0919202F09193023097A9F09C
:1022D00080910001882359F08091650187FF07C034
:1022E000809197018093980186E080939701028006
:1022F000F381E02D87E991E0099508952091EF01A0
:10230000809582238093EF01982F977099F430E0A5
:10231000482F082E000C550B2417350759F09091C3
:10232000660192FF07C08595859585950E94AA173D
:102330001092EF0108959091660192FB222720F9F7
:10234000281779F080FB92F99093660160916501FE
:102350007091660184E090E00E94681C82E00E9417
:102360007E1108958091EE019091BD01891719F0B9
:102370008F5F8770FBCF08950F931F93CF93DF93E9
:102380008091BC0182958F7009F05AC08091B9018B
:10239000882309F455C08091EE011091BD01609130
:1023A000B7017091B801C091BA01D091BB0191E021
:1023B0006F3F09F090E0292F06E0811709F440C033
:1023C000209721F07F3F21F030E003C031E001C0D1
:1023D000322F90E030FD31C0089FF001099FF00DD1
:1023E0001124DF01A254BE4F11963C91119737136F
:1023F00024C03C91361321C012963C9112973111A2
:102400001CC013964D915C9114974C1B5D0B483C7E
:10241000510598F48091BC018F7080618093BC015C
:10242000ED53FE4F80818F708061808387EB91E058
:102430000E9480030E94B21103C001968770BDCF35
:10244000DF91CF911F910F910895A1E1B0E0EBE2F0
:10245000F2E10C94921C8C0185E0F801DE011D96DE
:1024600001900D928A95E1F7F801E2809091B70111
:102470006091B8014091BA015091BB0141155105DD
:1024800031F06F3F31F481E09F3F19F403C081E0E8
:1024900001C080E0F82FF1709F2E80FD1BC1F80174
:1024A00030812181C380D48087EBA82E81E0B82EB3
:1024B000F090B901F601E41BF50BFF2009F4C7C049
:1024C0008091BC01E83CF10508F092C0482F407FA4
:1024D00009F051C0621311C093130FC0FE2CE1101C
:1024E0000CC08F7080618093BC01C5010E94800385
:1024F0008091BC01F80185832AC1C114D10431F057
:102500002F3F31F481E03F3F19F403C081E001C067
:1025100080E080FD03C081E08E2502C080E090E075
:10252000F82FF170FF2E80FF1CC08091EE014091CA
:10253000BD0156E0841709F4E8C090E0589FF0010F
:10254000599FF00D1124E254FE4F6181261306C0FD
:102550006081631303C06281E61203C00196877035
:10256000E9CFFE2CEE2009F4F2C08091BC0181601D
:102570008093BC0149C0621306C0931304C0E110EC
:1025800002C0F80186C0C8010E94C617882351F115
:10259000EE2041F12091BC01822F82958F7090E056
:1025A000029774F08091B7019091B80198878F835A
:1025B0001986DB86CA862C87CE0107960E94800387
:1025C00086E0F801A7EBB1E001900D928A95E1F762
:1025D0000E94BC110AC06217C9F0C8010E94C61748
:1025E00081111EC0C8010E948003FF24F394AFC074
:1025F000482F407F81F787EB91E00E94800386E0BF
:10260000F50111928A95E9F7F12CA1C09313E5CF5A
:10261000E110E3CFF8018583C8010E94800354C014
:10262000EE2001F32091BC01822F82958F7090E003
:10263000029734F28091B7019091B8019A8389830F
:102640001B82DD82CC822E83CE010196B7CFE83C7F
:10265000F105D0F5FE2CEE2029F2621327C093136A
:1026600025C02091BC0120FD18C0822F82958F705B
:10267000482F50E04115510581F0F80125834F3076
:10268000510541F08F5F982F9295907F822F8F7028
:10269000892B8583C8010E94800386E0F801A7EB9F
:1026A000B1E001900D928A95E1F751C0C8010E94F6
:1026B000C617811185CF8091BC0181608093BC01D8
:1026C000C8010E94800343C086E0F50111928A95FB
:1026D000E9F73DC0EE2009F485CFC8010E94C61776
:1026E000F82E882309F47ECF86E0F801A7EBB1E04D
:1026F00001900D928A95E1F78091B7019091B80110
:102700000E9431170E94BC1122C03D872E878D8503
:102710009E850E943117292F22952F70223028F490
:102720009F7039F0811105C00BC0243028F49F70D0
:1027300049F4805E883020F0C8010E9480039F2CFD
:10274000F92C05C0F8019581907F99F7F9CF8F2D6D
:102750006196EBE00C94AE1CACE2B0E0E2EBF3E18E
:102760000C948B1C85B7806885BF85B7806885BF52
:1027700084B7877F84BF0FB6F894A89580916000D6
:10278000886180936000109260000FBE90E080E846
:102790000FB6F89480936100909361000FBE84E5BA
:1027A0009EE090936301809362010E94D30C0E948B
:1027B000F20C8091E20084608093E2007894809132
:1027C0008C018823A1F01091E9001F709091EC001A
:1027D000892F817090FD80E8182B1092E90080917C
:1027E000E80083FD0E94C4091F701093E90082E095
:1027F00084BD93E095BD9DE797BD80936E000E94D8
:10280000231C811102C00E94131C0DE411E0D801A9
:102810008D918D018F3F11F00E94990EB1E0093525
:102820001B07A9F709E511E0F80181918F018F3F9E
:1028300011F00E94990EF1E002361F07A9F788E116
:10284000EBE4F2E0DF01282F1D922A95E9F7E6E19B
:10285000F2E0DF011D928A95E9F780E090E00E94A6
:10286000441C873E9E4F21F40E94231C811161C0AD
:1028700067EE7EEF80E090E00E94681C60E082E0FE
:1028800090E00E944A1C60E083E090E00E944A1CB5
:1028900010922E0260E074E184E090E00E94681CD7
:1028A00060E086E090E00E944A1C6FEF87E090E0D5
:1028B0000E944A1C40E050E0BA0188E090E00E948B
:1028C0005C1C60E08DE090E00E944A1C40E050E01B
:1028D000BA0188E190E00E945C1C60E087E190E032
:1028E0000E944A1C40E050E0BA018CE190E00E9456
:1028F0005C1C60E070E080E290E00E94681C40E0B8
:1029000050E0BA0188E190E00E945C1C80E00E94E7
:10291000F41B0E94131C40E050E0BA018FE090E0ED
:102920000E945C1C40E050E0BA0183E190E00E940C
:102930005C1C82E090E00E943C1C8093310284E0A9
:1029400090E00E94441C90936601809365010E9470
:10295000B00EEFE1FEE43197F1F700C000000E94F5
:10296000B00E80914B0280FF08C06FEF7FEF80E0D8
:1029700090E00E94681C0E94A11983E090E00E94F0
:102980003C1C0E94C31781E091E0909393028093D6
:1029900092028E010F5F1F4FCE0149969CA78BA715
:1029A00080918C01853009F047C062E0F62E80915D
:1029B0008C01853009F03CC080918C01843021F17C
:1029C00010929602A8E1B0E0E0E40FB6F894A89562
:1029D000A09360000FBEE093600083B7817F8460A6
:1029E00083BF83B7816083BF7894889583B78E7FD8
:1029F00083BF0FB6F894A89580916000886180939A
:102A00006000109260000FBE80918B01882309F452
:102A1000CECF0E94B00EEBE4F2E081919191892B30
:102A200009F0D1C183E692E08E179F07B1F7BFCFBF
:102A30000E94FD170E94D31A0E94B00E42E3C42EDA
:102A400042E0D42E5BE4E52E52E0F52E2AE432E09B
:102A5000D701F601419151918D919D918427952740
:102A60002E173F0719F0892BA9F322C0892B01F5F6
:102A70000E94F7196C0180912F0290913002C816C4
:102A8000D90609F457C08FEF89A38AA31BA20E941D
:102A9000F7198160782F9DA38CA349A15AA16BA13E
:102AA0008DA10E94E302D0923002C0922F0242C058
:102AB0003BE4432E32E0532E312CD2018D909D9079
:102AC0002D01F601608071806824792461147104FD
:102AD00041F1212CAA24A394B12CC3018A219B216A
:102AE000892BB1F02EA23FA221E0C4018A219B21B3
:102AF000892B09F420E028A70E94F7198160782F1C
:102B00009AA789A74EA15FA168A58AA50E94E302A2
:102B10002394AA0CBB1CF9E02F12DFCFD6018D92B3
:102B20009C923394B2E0CB0ED11CECE03E12C5CFA8
:102B30000E94EB190E94D31A90914A02891721F042
:102B400080934A020E94EB1980918C01843009F035
:102B500027CF83E08093E9008091E80082FF20CFB7
:102B60008091E80085FF23C00E94210E81111DC0C5
:102B700080E2C82ED12CCE0101965C0109C0809163
:102B8000F100D5018D935D01B1E0CB1AD10869F058
:102B90008091E80085FDF3CF8091E8008B778093EA
:102BA000E8000E94210E882399F391E001C090E093
:102BB0008091E8008B778093E800992309F4F0CEA8
:102BC000E9818E2F90E0FC013197E331F10508F0A7
:102BD000F1C0EB56FF4F0C947E1C1A828BE055C05F
:102BE0008A81823009F405C150F4813009F0E2C0D5
:102BF0000E94EB199B838C837D836E83DDC08330C1
:102C000041F0843009F0D6C01B821C821D821E82D6
:102C1000D3C0FE013196D7018C9111969C91B2E000
:102C2000EB0EF11C9283838332968BA59CA58E17A5
:102C30009F0789F7C1C08A81823021F0853009F46D
:102C4000BBC0B8C06B817C818D819E810E94841C39
:102C50000E94EF1BB1C04C816B818A810E94C11B15
:102C60009D83CEC02D813E813227232732274C8180
:102C70006B818A810E94651B9FC00E948C1B9CC037
:102C800080E152C082E08A838AE28B8395C0EA8029
:102C9000FB80FE24EF24FE24AC80B12C6801C70128
:102CA0008A529E4F9601201B310B2A153B0508F0D6
:102CB00083C0AAE2EA16A2E0FA0628F40E943C1CAD
:102CC000F601848303C0D60114961C92BFEFEB1A61
:102CD000FB0AEFEFCE1ADE0AE2CFEA80FB80FE2489
:102CE000EF24FE24AC80B12C6801C7018A529E4FAC
:102CF0009601201B310B2A153B0508F05DC0FAE256
:102D0000EF16F2E0FF0628F4D60114966C910E94AB
:102D10004A1CBFEFEB1AFB0AEFEFCE1ADE0AE5CF33
:102D20000E94551B49C082E08A8346C0EA80FB802E
:102D3000FE24EF24FE24AC80B12C6801C7018696E6
:102D40009601201B310B2A153B05B0F5F0EBEF1671
:102D5000F1E0FF0630F40E943C1CD60114968C93DF
:102D600002C0F6011482FFEFEF1AFF0A2FEFC21A1A
:102D7000D20AE4CFEA80FB80FE24EF24FE24AC805C
:102D8000B12C6801C70186969601201B310B2A15CC
:102D90003B0590F4A0EBEA16A1E0FA0620F4F60158
:102DA00064810E944A1CFFEFEF1AFF0A2FEFC21A3C
:102DB000D20AE8CF8FEF898340E250E0B80182E089
:102DC0000E946319EDCD19BCF9BC09B400FEFDCF1A
:102DD0008091D8008F7D8093D8008091E000826040
:102DE0008093E0008091E00081FDFCCF0E94FD1700
:102DF000DECD85E290E00E943C1C1B821C821D827D
:102E00008E83DACFCF92DF92FF920F931F93CF93EF
:102E1000DF936C010091960180912E02082BC7E090
:102E2000D0E010E0C8010C2E02C0959587950A9459
:102E3000E2F780FD04C02197A8F7F12C09C0FC2E11
:102E4000B6018C2F0E94700F0E947E0F019799F39C
:102E50008F2DDF91CF911F910F91FF90DF90CF9039
:102E60000895CF93DF93EC010E940217BE010E94E8
:102E7000700F0E947E0FDF91CF910895292F9C3013
:102E800078F5893068F590E039E0239F800D911D39
:102E90001124682F677023E0969587952A95E1F7AE
:102EA000FC01EE0FFF1FE80FF91FED59FD4F40E049
:102EB00050E080E0219130E0062E02C03695279543
:102EC0000A94E2F721703327042E01C0220F0A94DE
:102ED000EAF7822B4F5F5F4F4330510559F7089552
:102EE00080E00895292F9C3088F5893078F590E0AE
:102EF00039E0239F800D911D1124282F277051E068
:102F000001C0550F2A95EAF723E0969587952A95F3
:102F1000E1F7FC01EE0FFF1FE80FF91FED59FD4F20
:102F200020E030E070E04081CB01022E02C0969597
:102F300087950A94E2F781708195842785238427F9
:102F400081932F5F3F4F2330310569F708958093B8
:102F50009601089521E030E001C0220F8A95EAF73A
:102F600020958091960182230E94A717089521E061
:102F700030E001C0220F8A95EAF780919601822BFA
:102F80000E94A717089580932E020895CF93FC0105
:102F90008081918123813481232B31F09F3F31F453
:102FA00091E08F3F19F403C091E001C090E0C92F78
:102FB000C17090FD1CC0808191810E943117929553
:102FC0009F70963079F010F4925001C09A50923070
:102FD00088F4803F71F018F4883E60F40AC0843FA2
:102FE00049F407C0883E28F0813F21F402C0C0E0C8
:102FF00001C0C1E08C2FCF910895109211028091F1
:103000000001882331F08091650187FF02C08EE1C5
:1030100001C086E0E9E9F1E0DF011D928A95E9F758
:1030200080E090E00E94AE1A80E090E00E94891A51
:10303000109210020E9429110895882321F00E9405
:1030400022110E9429110895882339F090911102CC
:10305000892B809311020E9429110895882309F475
:1030600055C0682F823869F40E94D31A81FF4EC080
:1030700069E387E991E00E94541A0E94291169E3EB
:103080000EC0833899F40E94D31A80FF3FC063E5D5
:1030900087E991E00E94541A0E94291163E587E9AB
:1030A00091E00E942C1A0E9429110895843869F435
:1030B0000E94D31A82FF2AC067E487E991E00E9448
:1030C000541A0E94291167E4EACF8CEF860F813AE7
:1030D00030F380E2860F883048F4677081E001C0E9
:1030E000880F6A95EAF70E942211DDCF8BE5860FE3
:1030F000833028F480E090E00E94AE1A0895685A68
:10310000693120F480E090E00E94891A0895CF93FD
:10311000882309F4B4C0C82F8238B1F40E94D31AAE
:1031200081FDADC069E387E991E00E94541A0E94D5
:1031300029112FEF83EF91E0215080409040E1F77B
:1031400000C0000069E317C08338E1F40E94D31A7D
:1031500080FD95C063E587E991E00E94541A0E94C2
:1031600029112FEF80E792E0215080409040E1F755
:1031700000C0000063E587E991E00E942C1A0E94DC
:1031800029117DC08438B1F40E94D31A82FD77C022
:1031900067E487E991E00E94541A0E9429112FEFF9
:1031A00080E792E0215080409040E1F700C00000AD
:1031B00067E4E1CF8CEF8C0F813AB8F58091000184
:1031C0008823E1F08091650187FF18C0EC2FE69518
:1031D000E695E695F0E0E956FE4F8281282F30E033
:1031E0004C2F477081E090E002C0880F991F4A95EC
:1031F000E2F782239323892B59F411C0E9E9F1E026
:103200008191C81729F021E0EF39F207C9F707C00B
:103210006C2F87E991E00E942C1A0E9429116C2FD3
:1032200087E991E00E94541AAACF80E28C0F88307F
:1032300068F4C77081E090E001C0880FCA95EAF792
:1032400090911102892B8093110299CFEBE5EC0F3D
:10325000E33040F4F0E0E85EFE4F808190E00E94B1
:10326000AE1A0DC0C85AC93150F4EC2FF0E0EE0F81
:10327000FF1FE55EFE4F808191810E94891ACF91E8
:1032800008951F93CF93DF93182F893319F0C0E06F
:10329000D0E002C0C0E5D0E0812F0E9487182097BF
:1032A00041F08FEC97E00197F1F700C00000219703
:1032B000F6CF812F0E942E18DF91CF911F91089594
:1032C0008091690108950F931F93CF93DF938B0132
:1032D000EA0190918C01943079F58F708093E90028
:1032E0008FEF9091E800815095FD06C09AE69A957F
:1032F000F1F700C08111F5CF8091E80085FF1CC077
:103300000E94210E882361F08091E8008E778093DF
:10331000E80012C0F80181918F018093F10021979C
:10332000209791F38091E80085FDF4CF8091E8002B
:103330008E778093E800E4CFDF91CF911F910F91BA
:10334000089581E08093E00080E28093D80010929D
:10335000C9008FE097E20197F1F700C0000087E015
:1033600090EBDC0180939B0290939C02A0939D02C2
:10337000B0939E029CE088E10FB6F894A8958093E4
:1033800060000FBE90936000FFCF78941F920F9261
:103390000FB60F9211248F939F93AF93BF93809199
:1033A000970290919802A0919902B0919A02019689
:1033B000A11DB11D8093970290939802A09399024A
:1033C000B0939A02BF91AF919F918F910F900FBED2
:1033D0000F901F9018952FB7F894609197027091F5
:1033E00098028091990290919A022FBF08952FB769
:1033F000F8948091970290919802A0919902B091CF
:103400009A022FBF08951F920F920FB60F921124A8
:103410008F939F93AF93BF9380919602811113C0B6
:103420008091970290919802A0919902B0919A028E
:103430004196A11DB11D8093970290939802A0938D
:103440009902B0939A02BF91AF919F918F910F9083
:103450000FBE0F901F901895209100012223C9F0F4
:103460002091650127FF15C0262F269526952695C4
:103470002E31C8F4FC01E20FF11D677081E090E08D
:1034800001C0880F6A95EAF780959281892382832B
:103490000895FC0106962281621301C012823196C2
:1034A000E817F907C1F70895209100012223C1F020
:1034B0002091650127FF14C0262F26952695269575
:1034C0002E3130F5FC01E20FF11D677081E090E0D4
:1034D00001C0880F6A95EAF79281892B828308954B
:1034E000FC0132962FEF30E04191641789F02F3FB5
:1034F00019F4411101C0232F3F5F3630A9F72F3F48
:1035000039F0FC01E20FF11D27FDFA956283089561
:103510000895A3E0B0E0EFE8FAE10C949B1C209141
:1035200094023091950228173907A1F090939502E3
:1035300080939402E0919202F0919302309751F0BF
:1035400024E029839B838A830680F781E02DCE01C6
:10355000019609952396E2E00C94B71CA3E0B0E035
:10356000E4EBFAE10C949B1C2091900230919102C3
:1035700028173907A1F09093910280939002E0916F
:103580009202F0919302309751F023E029839B83BC
:103590008A830680F781E02DCE0101960995239656
:1035A000E2E00C94B71CE0919202F0919302309704
:1035B00029F00190F081E02D0995089580E00895AB
:1035C0000F931F93CF93DF93C42F122FFC0182819F
:1035D0008823B1F040938F020E94F71990938E02D6
:1035E00080938D0280E28C0F883008F059C0C7703C
:1035F00081E001C0880FCA95EAF70E94241850C0E4
:1036000080918F0248133CC020918D0230918E0230
:103610004FB7F8948091970290919802A0919902E7
:10362000B0919A024FBF821B930B883C910540F5E5
:10363000D0E2D10FC117B9F080E28C0F883040F48E
:10364000C77081E001C0880FCA95EAF70E941D1873
:10365000D83018F581E0912F977001C0880F9A95A6
:10366000EAF70E942418802F0E944119D830C0F434
:10367000212F277081E001C0880F2A95EAF70AC040
:1036800080E28C0F883060F4C77081E001C0880F41
:10369000CA95EAF70E941D1803C0802F0E944119A5
:1036A000DF91CF911F910F910895CF93DF93C6EDD6
:1036B000D1E060E0CE010E944A1C2196C11584E051
:1036C000D807B9F7DF91CF9108951F93CF93DF9378
:1036D000962F8230E8F46C30D8F44930C8F4632F68
:1036E000122FC42FD0E0CC0FDD1F22E1929FC00D1E
:1036F000D11D112498ED899FC00DD11D1124CE013B
:1037000086960E944A1C612FCE0187960E944A1C11
:10371000DF91CF911F910895A0E0B0E0E2E9FBE1D5
:103720000C94931CA12CE12CF12CB12C00E010E0A6
:10373000C0E0D0E06701C00ED11EFE01EE0FFF1FFA
:10374000EC0DFD1DEA58FC4F259134914C2F6B2D4B
:103750008A2D0E94651B2196C930D10571F70E5E36
:103760001F4FB3948CE0B812E3CF88EDE80EF11C44
:10377000A39482E0A812D9CFCDB7DEB7EAE00C94CB
:10378000AF1C0F931F93CF93DF93823008F56C30FB
:10379000F8F44930E8F4C42FD0E0CC0FDD1F22E16B
:1037A000629FC00DD11D112438ED839FC00DD11D26
:1037B0001124CE0186960E943C1C90E0182F002711
:1037C000CE0187960E943C1C9801282BC90102C09B
:1037D00080E090E0DF91CF911F910F91089585E2F5
:1037E00090E00E944A1C0895CF93C82F811102C017
:1037F0006FEF01C062E282E290E00E944A1CC111B8
:1038000002C06FEF01C062E183E290E00E944A1CB7
:10381000C11102C06FEF01C068E084E290E00E9435
:103820004A1CCF91089580E00E94F41B60E070E094
:10383000CB010E94EF1B0E948C1B0E94551B81E054
:103840000E94F41B089582E290E00E943C1C8232A8
:1038500081F483E290E00E943C1C823151F484E2C6
:1038600090E00E943C1C91E0883009F090E0892FA4
:1038700001C080E081700895F999FECF92BD81BDAD
:10388000F89A992780B50895A8E1B0E042E050E0A9
:103890000C94701C262FF999FECF92BD81BDF89A29
:1038A000019700B4021639F01FBA20BD0FB6F89484
:1038B000FA9AF99A0FBE08950396272F0E944B1C7F
:1038C0000E944A1C252F0E944B1C242F0C944B1C39
:1038D0000196272F0E944B1C0C944A1CDC01CB0143
:1038E000FC01F999FECF06C0F2BDE1BDF89A319610
:1038F00000B40D9241505040B8F70895EE0FFF1FED
:103900000590F491E02D0994692796276927782777
:103910008727782708952F923F924F925F926F9258
:103920007F928F929F92AF92BF92CF92DF92EF924F
:10393000FF920F931F93CF93DF93CDB7DEB7CA1BD0
:10394000DB0B0FB6F894DEBF0FBECDBF09942A88FB
:10395000398848885F846E847D848C849B84AA84A3
:10396000B984C884DF80EE80FD800C811B81AA8130
:10397000B981CE0FD11D0FB6F894DEBF0FBECDBFFB
:10398000ED010895FB01DC0104C08D9101908019C7
:1039900021F441505040C8F7881B990B0895F894C2
:0239A000FFCF57
:1039A20001601994098C098D0940226D8F026D0204
:1039B2000002E102FA021A03818283E200E900EACC
:1039C20000B500B600B700CD008301CC008A019299
:1039D2000194012102230224022502260227022A3F
:1039E20002B300B4006F0070009F01CB019190936D
:1039F2009295306667F6F7F5F49496973435F1F0C0
:023A0200C636C6
:00000001FF
